:100000000C942A001895000018950000189500001F
:10001000189500001895000018950000189500002C
:10002000189500000C94C007189500001895000062
:10003000189500001895000018950000189500000C
:1000400018950000189500001895000018950000FC
:10005000189500008FE58DBFC0E2E8EB4E2E88E0DA
:100060008EBFD8E0F7E05F2EEEEFF7E0A0E6B0E05D
:1000700088278D933197E9F7662481E48ABB81E371
:100080008BBB8FEB87BB8FEB88BB88E184BB83E0A6
:1000900085BB80E081BB8BE382BB80E08FBD81E0CC
:1000A0008EBD8FE181BD87E181BDC398C29AD89A88
:1000B000DE9AC498C798C598AC9AF894A8950E94FF
:1000C000EF088091D30080628093D300EFEFF1E0DE
:1000D000A4ECB0E091E00E942D280091C400003013
:1000E00081E009F080E08F930091C4000E3F80E032
:1000F00010F009F081E09F91892B882311F40C9472
:1001000084008EEB8093C4000091C4004AE0040F89
:1001100001BF89E190E00E94F026EAE0F0E0BB2711
:10012000A0E10E942A28013311F40C94DF00EAE0D8
:10013000F0E0A0E1BB2781E38C937BE70E941928C4
:10014000EBE0F0E0A0E1BB278FE08C937BE70E941F
:100150001928ECE0F0E001E010E0A0E1BB277BE72C
:100160000E941B28EEE0F0E0A0E1BB2780E08C932A
:100170007BE70E941928E2E1F0E000E010E0A0E156
:10018000BB277BE70E941B28EFE0F0E0A0E1BB2744
:1001900080E08C937BE70E941928E0E1F0E0A0E189
:1001A000BB2780E08C937BE70E941928E1E1F0E017
:1001B000A0E1BB2780E08C937BE70E941928EBE04D
:1001C000F0E0AFEBB0E00E942A280091BF000436B7
:1001D00018F011F00C94EE000C94F10084E680937A
:1001E000BF0080ED97E8A0ECB0E08D939C93ECE02D
:1001F000F0E0AAEBB0E00E942C28EEE0F0E0A5ECE5
:10020000B0E00E942A28EFE0F0E0A6ECB0E00E9407
:100210002A280E94F308E0E1F0E0AFE6B0E00E9497
:100220002A28E1E1F0E0A0E7B0E00E942A28E2E11C
:10023000F0E0A3E6B0E00E942C28A3E6B0E00E9424
:10024000F125E2E1F0E0A3E6B0E07BE70E941B28A5
:10025000AAEBB0E00D911C91003050E0150711F0B1
:100260000C94380181E090E0AAEBB0E08D939C9370
:1002700080E08093D20080916C00877F80936C0037
:1002800080E08093C80086E08093C2008DE0809378
:10029000C300EBE6F0E0FA93EA930E94D5172296AA
:1002A00084E190E00E94F026DE980E94DC26C49A49
:1002B00088EC90E00E94F026A89581B5886181BD08
:1002C000877F81BDE0E6F0E0FA93EA930E94EB1BA2
:1002D0002296A89500916000003011F40C947601EC
:1002E0000E94331B0E94B6080C947B018091D300BE
:1002F0008F7B8093D3000E945C1B84E690E00E9479
:10030000F02600916B00003018F011F00C948A0177
:100310000C949101EBE6F0E0FA93EA930E94421903
:1003200022960027A3EDB0E08C9186FB0EF401E04D
:1003300040E0041711F00C949F010E94380F82E3F3
:1003400090E00E94F0267894A89581B5886081BDE0
:1003500000916F00003011F00C94B40181E090E046
:10036000AAEBB0E08D939C9300916F00013011F0E7
:100370000C94C601AAEBB0E00D911C9141E050E055
:10038000040F151FAAEBB0E00D931C93A6EBB0E091
:100390004D915C91AAEBB0E00D911C9104171507EB
:1003A00018F011F00C94D6010C94DC0181E090E07F
:1003B000AAEBB0E08D939C930027ACE6B0E08C9163
:1003C00084FB0EF401E041E0041781E009F080E0D5
:1003D0008F930027A3EDB0E08C9186FB0EF401E033
:1003E00040E0041781E009F080E09F918923882391
:1003F00011F40C940E02EAEBF0E0FA93EA935A92AD
:100400004A9280E0A42DB52D8C9381E00E94DE25D8
:100410000E94300D249681E00E94DA250091700040
:10042000023081E009F080E08F930027A3EDB0E077
:100430008C9186FB0EF401E040E0041781E009F0A6
:1004400080E09F918923882311F40C94470281B5A1
:10045000886181BD877F81BDE3E0F0E00E9467266F
:10046000EAEBF0E0FA93EA935A924A9280E0A42DE4
:10047000B52D8C9381E00E94DE250E94300D2496DC
:1004800081E00E94DA25A89581B5886081BD80E071
:100490008093BC0080E080936B0080916C008F772C
:1004A00080936C000027A3EDB0E08C9186FB0EF4E6
:1004B00001E041E0041711F00C9460020E94EF0883
:1004C000A895ADE6B0E088278C930091D20000306B
:1004D00081E009F080E08F930027ACE6B0E08C91DA
:1004E00081FB0EF401E040E0041781E009F080E0B8
:1004F0009F91892B882311F40C94FA03E0E6F0E035
:10050000FA93EA930E942D18229600916000003021
:1005100018F011F00C948E020C94FA0380916C0088
:10052000806880936C000091D400003011F00C942E
:10053000EA024091C80000916000041718F011F021
:100540000C94A4020C94EA02809160008093C8008D
:100550000027ACE6B0E08C9184FB0EF401E040E0B3
:10056000041711F00C94C402A0E6B0E08C91AAEB41
:10057000B0E08D9388278C93ADE6B0E0E0EBF0E53A
:100580000E9432270C94EA020027A3EDB0E08C9180
:1005900087FB0EF401E041E0041711F00C94E40233
:1005A000A0E6B0E00D91112741E050E0040F151FC7
:1005B000AAEBB0E00D931C93ADE6B0E0E0EBF0E504
:1005C0000E9432270C94EA02ADE6B0E0E2EBF0E5DF
:1005D0000E9432270091D400013011F00C946A037C
:1005E00000916000013011F00C94FC02ADE6B0E027
:1005F000E2EBF0E50E94322700916000023011F03A
:100600000C940803ADE6B0E0E4EBF0E50E9432277D
:1006100080E08093620000916000033081E009F087
:1006200080E08F930091BF00043681E008F080E005
:100630009F918923882311F40C942603AFEBB0E03B
:100640008C918E5F8C9381E08093620000916000BA
:10065000043081E009F080E08F930091BF00023008
:1006600080E010F009F081E09F918923882311F444
:100670000C944203AFEBB0E08C9182508C9381E0FC
:100680008093620000916200013011F00C946A03C3
:100690008EB5887F8EBD5A924A928091BF00A42D5C
:1006A000B52D8C9381E00E94DE250E944D2222967A
:1006B00081E00E94DA25EBE0F0E0AFEBB0E07BE711
:1006C0000E9419280091D200013011F00C946A03A5
:1006D00081E08EBD0091D400023011F00C94FA0339
:1006E0004091C80000916000041718F011F00C94BC
:1006F0007B030C94FA03809160008093C800009102
:100700006000013011F00C94910381E090E0AAEBBD
:10071000B0E08D939C93ADE6B0E0E0EBF0E50E9495
:10072000322700916000023011F00C94E203A6EB36
:10073000B0E00D911C91013050E0150718F011F058
:100740000C94A4030C94DC03A6EBB0E00D911C9177
:1007500041E050E0041B150BA3E6B0E00D931C93A1
:1007600001E010E00F931F93A3E6B0E08D919C9100
:100770008A939A930E940C262296402F512F1F9104
:100780000F91040F151FA5E6B0E00D931C93AAEB83
:10079000B0E04D915C91A5E6B0E00D911C9104177D
:1007A000150711F40C94B003A5E6B0E08D919C916F
:1007B000AAEBB0E08D939C93ADE6B0E0E0EBF0E502
:1007C0000E94322700916000033011F00C94EE0378
:1007D000ADE6B0E0E2EBF0E50E9432270091600068
:1007E000043011F00C94FA03ADE6B0E0E4EBF0E570
:1007F0000E9432270027ACE6B0E08C9184FB0EF417
:1008000001E041E0041781E009F080E08F930027C8
:10081000A3EDB0E08C9187FB0EF401E041E00417FA
:1008200081E009F080E09F9189238F930091D200AD
:10083000013081E009F080E09F918923882311F441
:100840000C946504AAEBB0E00D911C91013050E0CE
:10085000150711F00C946504E0E6F0E0FA93EA93D2
:100860000E942D18229600916000003080E010F068
:1008700009F081E08F93A6EBB0E04D915C91A0E68A
:10088000B0E00D9111270417150781E008F080E012
:100890009F918923882311F40C946504A0E6B0E0AD
:1008A0000D91112741E050E0040F151FAAEBB0E0B5
:1008B0000D931C93ADE6B0E0E0EBF0E50E9432272B
:1008C00080916C00806880936C000027ACE6B0E0FB
:1008D0008C9180FB0EF401E040E0041711F00C94C1
:1008E0001605EBE6F0E0FA93EA930E94D5172296FC
:1008F00000916B00043011F00C9485040E94A6084E
:1009000080916C00806880936C0000916B000130D6
:1009100011F00C949604ADE6B0E0E2EBF0E50E9435
:10092000322780916C00806880936C0080E0809317
:10093000600000916B00023081E009F080E08F934D
:100940000091BF00043681E008F080E09F91892388
:10095000882311F40C94B404AFEBB0E08C918B5F5E
:100960008C9381E08093600000916B00033081E004
:1009700009F080E08F930091BF00053081E009F01D
:1009800080E09F918923882311F40C94CD0481E0A9
:100990008093BF0081E08093600000916B00033082
:1009A00081E009F080E08F930091BF00053080E086
:1009B00010F009F081E09F918923882311F40C94B1
:1009C000E904AFEBB0E08C9185508C9381E080938B
:1009D000600000916000013011F00C9416058EB596
:1009E000887F8EBD5A924A928091BF00A42DB52D6A
:1009F0008C9381E00E94DE250E944D22229681E0A8
:100A00000E94DA25EBE0F0E0AFEBB0E07BE70E947C
:100A100019280091D200013011F00C94110581E0E9
:100A20008EBD80916C00806880936C00EDE6F0E0F4
:100A3000ADE6B0E00E943C27ADE6B0E08C9180309E
:100A400081E009F480E08F9300916B00003081E039
:100A500009F480E09F91892B8F930091BC000130B5
:100A600081E009F080E09F91892B882311F40C9498
:100A700052020091BC00013011F00C94600580E03E
:100A80008093BC00ADE6B0E0E2EBF0E50E943227D7
:100A90000027A3EDB0E08C9187FB0EF401E041E06C
:100AA000041711F00C94600581E090E0AAEBB0E02F
:100AB0008D939C93ADE6B0E0E0EBF0E50E94322729
:100AC000ADE6B0E0E0EBF0E50E94442811F00C94B4
:100AD000D2050091D200013011F00C9471050E94F2
:100AE000A608A6EBB0E04D915C91AAEBB0E00D91A9
:100AF0001C910417150718F011F00C94CD05002770
:100B0000A3EDB0E08C9186FB0EF401E040E0041709
:100B100011F00C949E05EAEBF0E0FA93EA935A92F6
:100B20004A9280E0A42DB52D8C9381E00E94DE25B1
:100B30000E94300D249681E00E94DA250027A3ED63
:100B4000B0E08C9186FB0EF401E041E0041711F057
:100B50000C94CB050E94B6080027A3EDB0E08C9161
:100B600086FB0EF401E040E0041711F00C94CB0575
:100B7000EAEBF0E0FA93EA935A924A9280E0A42DCD
:100B8000B52D8C9381E00E94DE250E94300D2496C5
:100B900081E00E94DA250C94D00580E08093C800A3
:100BA0000C94F206E2EBF0E50E94442811F00C945C
:100BB0006A060091D200013011F00C94E1050E9408
:100BC000A608AAEBB0E00E94F1250027A3EDB0E053
:100BD0008C9185FB0EF401E041E0041711F00C94B8
:100BE00006060027ACE6B0E08C9184FB0EF401E031
:100BF00040E0041711F00C940106AAEBB0E00E944B
:100C0000F8258091D3008F7D8093D300A6EBB0E0D0
:100C10004D915C91AAEBB0E00D911C910417150762
:100C200018F011F00C9416060C941C0681E090E06C
:100C3000AAEBB0E08D939C930027A3EDB0E08C91DC
:100C400086FB0EF401E040E0041711F00C943B0623
:100C5000EAEBF0E0FA93EA935A924A9280E0A42DEC
:100C6000B52D8C9381E00E94DE250E94300D2496E4
:100C700081E00E94DA250027A3EDB0E08C9186FB8D
:100C80000EF401E041E0041711F00C9468060E9494
:100C9000B6080027A3EDB0E08C9186FB0EF401E0CE
:100CA00040E0041711F00C946806EAEBF0E0FA93C8
:100CB000EA935A924A9280E0A42DB52D8C9381E05C
:100CC0000E94DE250E94300D249681E00E94DA25E4
:100CD0000C94F206E4EBF0E50E94442811F00C9429
:100CE000E2060091D200013011F00C9479060E94C6
:100CF000A608AAEBB0E00D911C91013050E0150759
:100D000018F011F00C9486060C948C06AAEBB0E057
:100D10000E94F8250C949406A6EBB0E08D919C916E
:100D2000AAEBB0E08D939C930027A3EDB0E08C91EB
:100D300086FB0EF401E040E0041711F00C94B306BA
:100D4000EAEBF0E0FA93EA935A924A9280E0A42DFB
:100D5000B52D8C9381E00E94DE250E94300D2496F3
:100D600081E00E94DA250027A3EDB0E08C9186FB9C
:100D70000EF401E041E0041711F00C94E0060E942B
:100D8000B6080027A3EDB0E08C9186FB0EF401E0DD
:100D900040E0041711F00C94E006EAEBF0E0FA935F
:100DA000EA935A924A9280E0A42DB52D8C9381E06B
:100DB0000E94DE250E94300D249681E00E94DA25F3
:100DC0000C94F206E6EBF0E50E94442811F00C9436
:100DD000F206ECE0F0E0AAEBB0E07BE70E941B2813
:100DE0000C94F20681E090E00E94F0260027ACE629
:100DF000B0E08C9187FB0EF401E040E0041718F09E
:100E000011F00C9405070C94BE0700916B000030A4
:100E100018F011F00C940E070C947507A895E0E6F5
:100E2000F0E0FA93EA930E94D517229600916000B1
:100E3000043011F00C9469070E94A60880E08093AA
:100E4000C8000E94F10885E090E00E94F02680E052
:100E500080936200E0E6F0E0FA93EA930E94D517EF
:100E60002296A2E6B0E08C918F5F8C9388E090E0B0
:100E70000E94F02600916000003081E009F080E0DF
:100E80008F9300916200043680E010F009F081E059
:100E90009F91892B882311F40C942A0700916200FA
:100EA000043618F011F00C9457070C94660781B5BE
:100EB000886181BD877F81BDE3E6F0E0FA93EA9324
:100EC0000E94A809229681B5886081BD80E0809348
:100ED000600081E090E00E94F02600916000003008
:100EE00011F00C940E070C94B4070091D40001305B
:100EF00011F00C94B00780E090E0A3E6B0E08D9391
:100F00009C93E0E6F0E0FA93EA930E942D18229673
:100F1000A3E6B0E00E94F125EF93FF93ECE8F1E047
:100F20000E94C426FF91EF9100916000003081E0A3
:100F300009F080E08F93A3E6B0E00D911C91083298
:100F400050E0150780E010F009F081E09F91892BB7
:100F5000882311F40C94810781E090E00E94F02630
:100F600081E090E00E94F0260091D200003011F064
:100F70000C94BE0785E090E00E94F0260C944D0290
:100F80000F921F922F923F924F925F927F92AF9259
:100F9000BF920F931F932F933F934F935F936F9342
:100FA0007F938F939F93AF93BF93CF93DF93EF93F1
:100FB000FF938FB78F93F89489B78B7F89BF8EB5D6
:100FC000887F8EBD5A924A9280E092E0A42DB52D82
:100FD0008D939C9382E00E94DE250E9458252296E4
:100FE00082E00E94DA250091DD000A3011F00C94B5
:100FF000FB070E94EF080E94C91E0091DD000A3025
:1010000011F00C9408080E94F10880E08093DD0044
:10101000ADEDB0E08C918F5F8C93A8950027A3ED88
:10102000B0E08C9186FB0EF401E040E0041711F073
:101030000C942D085A924A9280E092E0A42DB52D8E
:101040008D939C9382E00E94DE250E945825229673
:1010500082E00E94DA250E94C91EA9EDB0E04D9100
:101060005D916D917C91A5EDB0E00D911D912D915B
:101070003C910E94902780E00CF481E08F93002740
:10108000A3EDB0E08C9186FB0EF401E040E0041784
:1010900081E009F080E09F918923882311F40C946A
:1010A0005E0880E49CE990934D0080934C0081E0C1
:1010B0008EBD89B7846089BF0C94880880E08093D6
:1010C000D20080916C00877F80936C000027A3ED95
:1010D000B0E08C9186FB0EF401E040E0041711F0C3
:1010E0000C947B08ACE6B0E08C9184FBACEBB0E0F8
:1010F000882780F98C930091C5004FE70423A1E66F
:10110000B0E00C930E94F10880E08093C800AC9A94
:101110008F918FBFFF91EF91DF91CF91BF91AF91F1
:101120009F918F917F916F915F914F913F912F91FF
:101130001F910F91BF90AF907F905F904F903F9025
:101140002F901F900F901895F894FFCF89B78B7F41
:1011500089BF8EB5887F8EBD80E08093D20080915C
:101160006C00877F80936C00AC9A0895DE9A6E982D
:10117000C498C598C7980E94F108E2E0F0E00E9488
:101180006726DE98C49A0E94DC2684E690E00E94DE
:10119000F026A8958091D3008F7B8093D300E0E662
:1011A000F0E0FA93EA930E94EB1B22960091600014
:1011B000003011F40C94EC088091D300806480938B
:1011C000D30084E690E00E94F026DE9A6E98C498E0
:1011D000C598C7980C94EE080E94380F0895AB98F4
:1011E0000895AB9A089581E00E94FF2680916C00DB
:1011F0008F7E80936C000091C50041E00423A8819C
:10120000B9810C93A881B9810C91003011F40C9430
:101210000E0980916C00806180936C008091D300F6
:101220008F778093D3000091C50042E00423A8810A
:10123000B9810C93A881B9810C91003011F40C9400
:1012400026098091D30080688093D30080916C0040
:101250008E7F80936C000091C50044E00423A88138
:10126000B9810C93A881B9810C91003011F40C94D0
:101270003E0980916C00816080936C0080916C00CD
:101280008D7F80936C000091C50048E00423A88105
:10129000B9810C93A881B9810C91003011F40C94A0
:1012A000560980916C00826080936C0080916C0084
:1012B0008F7D80936C000091C50040E20423A881DB
:1012C000B9810C93A881B9810C91003011F40C9470
:1012D0006E0980916C00806280936C008091D300D5
:1012E0008F7E8093D3000091C60041E00423A88143
:1012F000B9810C93A881B9810C91003011F40C9440
:1013000086098091D30080618093D3000091C6004C
:1013100046E00423A881B9810C93A881B9810C917E
:1013200042E00E9434280C93A881B9818C9180936B
:10133000D4000091D400033011F00C94A20982E093
:101340008093D40081E0481A8827580A229608958D
:1013500082E00E94FF2681E00E94FF2681E00E9439
:10136000FF2680E0AA81BB818C9383E4A0EAB0E0F1
:101370008C938FE4A1EAB0E08C938EE4A2EAB0E013
:101380008C9386E4A3EAB0E08C9389E4A4EAB0E00D
:101390008C93ACE6B0E08C9185FBA881B98188275D
:1013A00080F98C9380916C00806280936C00A6E73A
:1013B000B0E00D911D912D913C91A6E9B0E00D9307
:1013C0001D932D933C935A924A92A6E9B0E00D9159
:1013D0001D912D913C91A42DB52D0D931D932D9311
:1013E0003C9384E00E94DE255A924A9280E090E08D
:1013F000A42DB52D8D939C9382E00E94DE255A92F8
:101400004A9281E0A42DB52D8C9381E00E94DE25C7
:101410000E944710269687E00E94DA258FE00E94FE
:10142000FF26E8EAF0E006E0A881B9810E940B28D7
:10143000A881B981E8EBF0E50E9444280FB68FE05F
:10144000481A8827580A22960FBE81E009F080E0EA
:101450008F9300919100003181E009F080E09F912D
:101460008923882311F40C94830A81E0AA81BB812B
:101470008C93A6E9B0E00D911D912D913C91A6E7CA
:10148000B0E00D931D932D933C9380916C008F7D64
:1014900080936C005A924A92A6E9B0E00D911D919A
:1014A0002D913C91A42DB52D0D931D932D933C931F
:1014B00084E00E94DE255A924A9280E090E0A42DBA
:1014C000B52D8D939C9382E00E94DE255A924A921C
:1014D00080E0A42DB52D8C9381E00E94DE250E9432
:1014E0004710269687E00E94DA25A6E9B0E00D9124
:1014F0001D912D913C91A6E7B0E00D931D932D9386
:101500003C930E94DD0AA881B9818C9180FBACE6F6
:10151000B0E08C9185F98C93AAE7B0E00D911D9114
:101520002D913C91A6E7B0E00D931D932D933C9334
:10153000A6E7B0E00D911D912D913C91A6E9B0E098
:101540000D931D932D933C935A924A92A6E9B0E0D5
:101550000D911D912D913C91A42DB52D0D931D93B1
:101560002D933C9384E00E94DE255A924A9280E0BB
:1015700090E0A42DB52D8D939C9382E00E94DE25F2
:101580005A924A9280E0A42DB52D8C9381E00E945E
:10159000DE250E944710269687E00E94DA25AA8160
:1015A000BB818C91AE81BF818D9388278C9384E021
:1015B000481A8827580A2696089582E00E94FF2636
:1015C00081E00E94FF2681E00E94FF26789481E05E
:1015D00090E0AC81BD818D939C93EA81FB81FA936D
:1015E000EA93EE81FF81FA93EA930E94F30C24962A
:1015F000AA81BB810C91013011F00C940A0B82E09E
:1016000090E0AC81BD818D939C9381E08093C50077
:101610000C94260B023011F00C94190B83E090E02F
:10162000AC81BD818D939C9380E08093C5000C9428
:10163000260B033011F00C94260B84E090E0AC8173
:10164000BD818D939C9383E08093C500EEE0F0E034
:10165000A5ECB0E07BE70E941928EC81FD81FA93AC
:10166000EA935A924A9280E0A42DB52D8C9381E0A2
:101670000E94DE250E94300D249681E00E94DA252A
:101680000091D200003011F00C94400B88EC90E0F7
:101690000E94F02685E090E0AC81BD818D939C9303
:1016A000EA81FB81FA93EA93EE81FF81FA93EA9350
:1016B0000E94F30C2496EEE0F0E0A5ECB0E00E946E
:1016C0002A28AA81BB810C91033011F00C946A0B7B
:1016D0000C94070CAA81BB810C91013011F00C9481
:1016E000780BA5ECB0E08C9188608C930C94810B06
:1016F000023011F00C94810BA5ECB0E08C91877F47
:101700008C93EEE0F0E0A5ECB0E07BE70E941928B6
:1017100088EC90E00E94F02686E090E0AC81BD81EC
:101720008D939C93EA81FB81FA93EA93EE81FF818A
:10173000FA93EA930E94F30C2496AA81BB810C9140
:10174000033011F00C94A60B0C94070CEEE0F0E0C3
:10175000A5ECB0E00E942A28AA81BB810C9101303F
:1017600011F00C94BA0BA5ECB0E08C9184608C93D2
:101770000C94C30B023011F00C94C30BA5ECB0E039
:101780008C918B7F8C93EEE0F0E0A5ECB0E07BE7F2
:101790000E94192888EC90E00E94F02687E090E0F3
:1017A000AC81BD818D939C93EA81FB81FA93EA938E
:1017B000EE81FF81FA93EA930E94F30C2496EEE007
:1017C000F0E0A5ECB0E00E942A28AA81BB810C9130
:1017D000013011F00C94F30BA5ECB0E08C91806219
:1017E0008C930C94FC0B023011F00C94FC0BA5ECC8
:1017F000B0E08C918F7D8C93EEE0F0E0A5ECB0E052
:101800007BE70E94192888EC90E00E94F02688E08F
:1018100090E0AC81BD818D939C93EC81FD81FA9326
:10182000EA930E94D10C22960091C50043E0042364
:10183000A881B9810C93A881B9810C91003011F075
:101840000C942A0C83E090E0AC81BD818D939C9335
:101850000C94400C013011F00C94360C82E090E0B6
:10186000AC81BD818D939C930C94400C033011F09E
:101870000C94400C84E090E0AC81BD818D939C93EE
:10188000EC81FD81FA93EA930E94D10C229600919B
:10189000C50048E00423A881B9810C93A881B981CF
:1018A0000C91003011F00C945D0C8AE090E0AC815A
:1018B000BD818D939C930C94670C083011F00C94AF
:1018C000670C89E090E0AC81BD818D939C93EC81A5
:1018D000FD81FA93EA930E94D10C22960091C500F3
:1018E00044E00423A881B9810C93A881B9810C91AB
:1018F000003011F00C94840C8BE090E0AC81BD8141
:101900008D939C930C948E0C043011F00C948E0CDF
:101910008CE090E0AC81BD818D939C93EC81FD8146
:10192000FA93EA930E94D10C22960091C50040E2FE
:101930000423A881B9810C93A881B9810C9100304E
:1019400011F00C94AB0C8DE090E0AC81BD818D93D7
:101950009C930C94B50C003211F00C94B50C8EE0F5
:1019600090E0AC81BD818D939C93EC81FD81FA93D5
:10197000EA930E94D10C22968FE090E0AC81BD8169
:101980008D939C93EC81FD81FA93EA930E94D10C94
:1019900022960E94F30884E0481A8827580A26965F
:1019A0000895E881F981FA93EA935A924A9280E085
:1019B000A42DB52D8C9381E00E94DE250E94300D70
:1019C000249681E00E94DA2582E390E00E94F026CE
:1019D0000091D200003011F00C94E80C82E390E00A
:1019E0000E94F026089581E00E94FF26EA81FB8193
:1019F000FA93EA935A924A9280E0A42DB52D8C93E3
:101A000081E00E94DE250E94300D249681E00E9434
:101A1000DA2584E690E00E94F026E881F981FA93C5
:101A2000EA930E94D5172296A881B9810C910030C3
:101A300018F011F00C941E0D0C940D0D0E94A608C8
:101A400084E190E00E94F026A881B9818C91AC815C
:101A5000BD818C9381E0481A8827580A2296089500
:101A600082E00E94FF2681E00E94FF268EB5887FDB
:101A70008EBD80916C00877F80936C00A6E7B0E0FC
:101A80000D911D912D913C91A6E9B0E00D931D9310
:101A90002D933C935A924A92A6E9B0E00D911D9184
:101AA0002D913C91A42DB52D0D931D932D933C9319
:101AB00084E00E94DE255A924A92AA85BB858D91C8
:101AC0009C91A42DB52D8D939C9382E00E94DE25E0
:101AD0005A924A9280E0A42DB52D8C9381E00E9409
:101AE000DE250E944710269687E00E94DA2540E016
:101AF00050E060E070E0A2E9B0E00D911D912D9101
:101B00003C910E94902711F00C94880D0C94320F98
:101B10000E9401225A924A928091BF00A42DB52DB5
:101B20008C9381E00E94DE250E944D22229681E066
:101B30000E94DA255A924A92A0ECB0E08D919C91D5
:101B4000A42DB52D8D939C9382E00E94DE250E94EA
:101B5000E522229682E00E94DA25AC98A6E9B0E060
:101B60000D911D912D913C91A5EDB0E00D931D932C
:101B70002D933C93A6E9B0E00D911D912D913C91E0
:101B8000A2E9B0E04D915D916D917C910E94862714
:101B9000A9EDB0E00D931D932D933D9380E0A881B6
:101BA000B9818C930E94C91E81E090E0AA81BB811B
:101BB0008D939C93AA81BB810D911C910F3F51E0A5
:101BC000150718F011F00C94140EAA81BB81AD908A
:101BD000BC90ADEDB0E0AA0DBB1D0C910F3F81E0B4
:101BE00009F080E08F93AA81BB81AD90BC90AEEDEF
:101BF000B0E0AA0DBB1D0C910F3E80E010F009F083
:101C000081E09F918923882311F40C940D0E81E0CB
:101C1000A881B9818C930C94140EAA81BB810E9477
:101C2000F12510F40C94DA0DA881B9810C910130E2
:101C300011F00C94D20DAA81BB81AD90BC90AFED98
:101C4000B0E0AA0DBB1D8C91AA81BB818D93882722
:101C50008C93AA81BB810D911C9140E150E00E94C0
:101C60004626AA81BB814D935C9380E18093C70097
:101C7000AA81BB810D911C91013050E0150711F034
:101C80000C94470E84E08093C7000C94D40E02306D
:101C900050E0150711F00C94520E85E08093C700B8
:101CA0000C94D40E033050E0150711F00C945D0E27
:101CB00086E08093C7000C94D40E043050E01507E2
:101CC00011F00C94680E87E08093C7000C94D40E3A
:101CD000053050E0150711F00C94730E88E08093E6
:101CE000C7000C94D40E063050E0150711F00C9488
:101CF0007E0E8AE08093C7000C94D40E073050E02B
:101D0000150711F00C94890E8CE08093C7000C9499
:101D1000D40E083050E0150711F00C94940E8EE0AC
:101D20008093C7000C94D40E093050E0150711F0D1
:101D30000C949F0E80E18093C7000C94D40E0A305F
:101D400050E0150711F00C94AA0E84E18093C700AF
:101D50000C94D40E0B3050E0150711F00C94B50E16
:101D600088E18093C7000C94D40E0C3050E0150726
:101D700011F00C94C00E8CE18093C7000C94D40E2B
:101D80000D3050E0150711F00C94CB0E80E28093DB
:101D9000C7000C94D40E0E3050E0150711F00C94CF
:101DA000D40E88E28093C700A2E9B0E00D911D91A6
:101DB0002D913C9140E052E060E070E00E940F27DE
:101DC000A7E6B0E00D931D932D933D93A7E6B0E0F9
:101DD0000D911D912D913C91A7ECB0E04C915527B0
:101DE000662777270E947026A7E6B0E04D935D93A3
:101DF0006D937D93A7E6B0E00D911D912D913C91DF
:101E000048EE53E060E070E00E947026A7E6B0E084
:101E10004D935D936D937D93AC81BD810C910030AA
:101E200011F00C94320F00916F00013011F00C94FE
:101E3000200FECE0F0E0AAEBB0E07BE70E941B286B
:101E400081E08093D20088EC9FEA90934D008093CC
:101E50004C0089B7846089BF81E08EBD85E090E049
:101E60000E94F02683E0481A8827580A249608958D
:101E7000A895A6E7B0E00D911D912D913C91AAE7A0
:101E8000B0E00D931D932D933C93A6E7B0E00D9128
:101E90001D912D913C91A6E9B0E00D931D932D93DA
:101EA0003C935A924A92A6E9B0E00D911D912D9172
:101EB0003C91A42DB52D0D931D932D933C9384E05F
:101EC0000E94DE255A924A9280E090E0A42DB52D22
:101ED0008D939C9382E00E94DE255A924A9280E084
:101EE000A42DB52D8C9381E00E94DE250E94471021
:101EF000269687E00E94DA25A895A6EBB0E00D9122
:101F00001C91013050E0150710F00C94AE0F5A925E
:101F10004A9281E0A42DB52D8C9381E00E94DE25AC
:101F20000E943F23229681E00E94DA258CE291E014
:101F30000E94F0265A924A9280E0A42DB52D8C93EF
:101F400081E00E94DE250E943F23229681E00E94CC
:101F5000DA258091D30080648093D300A895A6E70A
:101F6000B0E00D911D912D913C91A6E9B0E00D934B
:101F70001D932D933C93AAEBB0E00D911C91003082
:101F800050E0150781E009F080E08F93A6EBB0E008
:101F90004D915C91AAEBB0E00D911C9104171507CF
:101FA00080E010F009F081E09F91892B882311F4E3
:101FB0000C94E00F81E090E0AAEBB0E08D939C934D
:101FC0000E94F108089584E00E94FF26A5EDB0E08C
:101FD0000D911D912D913C91A881B9810D931D9377
:101FE0002D933C93A6E7B0E00D911D912D913C916E
:101FF000A6E9B0E00D931D932D933C935A924A921B
:10200000A6E9B0E00D911D912D913C91A42DB52D27
:102010000D931D932D933C9384E00E94DE255A92EC
:102020004A928FE19EE4A42DB52D8D939C9382E07E
:102030000E94DE255A924A9280E0A42DB52D8C9301
:1020400081E00E94DE250E944710269687E00E94CC
:10205000DA25A6E7B0E00D911D912D913C91A6E9FE
:10206000B0E00D931D932D933C93A881B9810D9100
:102070001D912D913C91A5EDB0E00D931D932D93F5
:102080003C9384E0481A8827580A2296089581E0F4
:102090000E94FF2681E00E94FF2681E00E94FF2629
:1020A00080E090E0A8EBB0E08D939C9380916C0071
:1020B0008F7B80936C0000E010E020E030E0A2E92C
:1020C000B0E00D931D932D933C930027ACE6B0E058
:1020D0008C9185FB0EF401E041E0041781E009F0EA
:1020E00080E08F93A885B9850D911C91003050E058
:1020F000150781E009F480E09F9189238F93AE81D9
:10210000BF810C91003081E009F080E09F9189232C
:10211000882311F40C94E710AAE9B0E0E885F9856A
:102120000E94A327EAE9F0E0A0EAB7E00E94FF27B7
:10213000E0EAF7E0AAE9B0E01127222704E033271C
:102140000E94482781E4AC81BD818C93AC81BD8124
:102150008C918093A00081E0EAE9F0E001E00A932D
:10216000ADE6B0E00E940428ADE6B0E08C91A1EAB3
:10217000B0E08C9382E0EAE9F0E001E00A93ADE69A
:10218000B0E00E940428ADE6B0E08C91A2EAB0E095
:102190008C9383E0EAE9F0E001E00A93ADE6B0E079
:1021A0000E940428ADE6B0E08C91A3EAB0E08C93E5
:1021B00084E0EAE9F0E001E00A93ADE6B0E00E94D5
:1021C0000428ADE6B0E08C91A4EAB0E08C9389B726
:1021D0008B7F89BF8EB5887F8EBD81B5886181BDBB
:1021E000877F81BDAEECB0E00D911D912D913C91AA
:1021F000AAECB0E00D931D932D933C93AAE7B0E0B9
:102200004D915D916D917C91A6E7B0E00D911D918E
:102210002D913C910E94902711F00C94191102E02D
:1022200010E020E030E0AAECB0E00D931D932D9378
:102230003C9380E0A881B9818C93EA81FB81FA9379
:10224000EA935A924A92AE85BF850D911D912D91C8
:102250003C91A42DB52D0D931D932D933C9384E0BB
:102260000E94DE250E949220249684E00E94DA25B6
:10227000AA81BB810C910E3F11F40C944B118091FB
:10228000D30080648093D30080916C00806480933D
:102290006C000C945E115A924A92AA85BB858D916E
:1022A0009C91A42DB52D8D939C9382E00E94DE25F8
:1022B0000E946112229682E00E94DA25A881B981EB
:1022C0008C918F5F8C9340917300A881B9810C91A0
:1022D000041781E009F080E08F930027ACE6B0E0BE
:1022E0008C9186FB0EF401E041E0041781E009F4D3
:1022F00080E09F918923882311F40C94141200919B
:1023000082000B3011F00C94C111EAECF0E0FA936A
:10231000EA935A924A92AAECB0E00D911D912D9148
:102320003C91A42DB52D0D931D932D933C9384E0EA
:102330000E94DE250E947916249684E00E94DA2508
:10234000EA85FB85FA93EA935A924A92AAECB0E0A6
:102350000D911D912D913C91A42DB52D0D931D93A3
:102360002D933C9384E00E94DE250E940F16249654
:1023700084E00E94DA2580E0A881B9818C930C94D6
:102380001212AAE7B0E04D915D916D917C91A6E7A4
:10239000B0E00D911D912D913C910E94902711F07C
:1023A0000C94D811AA85BB850E94E2250C941212C8
:1023B000EAECF0E0FA93EA935A924A92AAECB0E07F
:1023C0000D911D912D913C91A42DB52D0D931D9333
:1023D0002D933C9384E00E94DE250E94791624967A
:1023E00084E00E94DA25EA85FB85FA93EA935A9203
:1023F0004A92AAECB0E00D911D912D913C91A42D33
:10240000B52D0D931D932D933C9384E00E94DE2502
:102410000E940F16249684E00E94DA2580E0A881AD
:10242000B9818C930C941812AA85BB850E94E22571
:102430000027ACE6B0E08C9186FB0EF401E041E0B1
:10244000041711F00C941D11C49AA885B9850D913B
:102450001C91003050E0150711F00C943712A8EBD6
:10246000B0E08D919C91A6EBB0E08D939C93009190
:10247000D200013081E009F080E08F930027A3EDC6
:10248000B0E08C9186FB0EF401E040E0041781E09F
:1024900009F080E09F918923882311F40C945B124A
:1024A00080E593EC90934D0080934C0081E08EBDCD
:1024B00089B7846089BF83E0481A8827580A26961E
:1024C000089584E00E94FF2684E00E94FF2681E0B8
:1024D0000E94FF2681E00E94FF2681E00E94FF26E5
:1024E00081E00E94FF2680E0AE81BF818C93AE81A7
:1024F000BF810C910F3018F011F00C941C1481E086
:10250000AC81BD818C93AC81BD810C910C3018F0F5
:1025100011F00C94A3128FEF0E94E3260E94E5268F
:102520000E94E426AC81BD81AD90BB24A4E8B0E05C
:10253000AA0DBB1D8C93AC81BD818C918F5F8C9358
:1025400010F40C9483128DE0AC81BD818C93AC812E
:10255000BD810C91043118F011F00C94C1128FEF71
:102560000E94E3260E94E5260E94E426A881B98104
:102570008C93AC81BD818C918F5F8C9310F40C9403
:10258000A712EA85FB85FA93EA93EA85FB85FA931D
:10259000EA930E94A41424960027ACE6B0E08C9144
:1025A00086FB0EF401E041E0041711F00C94DA12FE
:1025B0000C94141480E0AA81BB818C93009190004C
:1025C000003281E009F080E08F93009190000031AB
:1025D00081E009F080E09F91892B882311F40C940D
:1025E000F51281E0AA81BB818C93009185000030B7
:1025F00081E009F480E08F9300918500053E81E041
:1026000009F480E09F9189238F93AA81BB810C916B
:10261000013081E009F080E09F918923882311F443
:102620000C94091400919000003211F00C941C13CA
:10263000A8EBB0E00E94F1250027ACE6B0E08C9159
:1026400085FB0EF401E040E0041711F00C945113E7
:1026500081E0AC81BD818C93AC85BD854D915C9151
:10266000A8EBB0E00D911C910417150781E009F06B
:1026700080E08F93A8EBB0E00D911C91003050E00A
:10268000150780E010F009F081E09F9189238823ED
:1026900011F40C944F1380E0AC81BD818C930C94A9
:1026A000851380E0AC81BD818C9381E0A881B981E4
:1026B0008C93A881B9810C91053018F011F00C941D
:1026C0008513A881B981AD90BB24AFE9B0E0AA0D14
:1026D000BB1D4C91A881B981AD90BB24A4E8B0E0AA
:1026E000AA0DBB1D0C91041711F40C947D1381E00D
:1026F000AC81BD818C930C948513A881B9818C9198
:102700008F5F8C9310F40C945913AC81BD810C91A4
:10271000003081E009F080E08F93AC85BD850D919C
:102720001C910F315EE4150781E009F080E09F9174
:10273000892B882311F40C9409140E943614A8855F
:10274000B9850D911D912D913C9140E052E060E0E2
:1027500070E00E947026A2E9B0E04D935D936D9306
:102760007D93E6E9F0E0FA93EA935A924A92AE85B5
:10277000BF850D911D912D913C91A42DB52D0D93EB
:102780001D932D933C9384E00E94DE250E940F163A
:10279000249684E00E94DA25809190008093910035
:1027A000AC85BD850D911C910F315EE4150711F0CC
:1027B0000C94DA13AC81BD810C91003011F00C94B3
:1027C000091480916C00806480936C0000919100EA
:1027D000003181E009F080E08F93AC85BD850D91DB
:1027E0001C910F315EE4150781E009F480E09F91B0
:1027F0008923882311F40C940914AA85BB850D91B3
:102800001D912D913C91AEECB0E00D931D932D9355
:102810003C9300918500003011F00C9414148091C9
:102820006C00806480936C00AE81BF818C918F5F5F
:102830008C9310F40C9477128FEF0E94E3260E9481
:10284000E5260E94E426A0E6B0E08C938FEF0E947C
:10285000E3260E94E5260E94E426A0E6B0E08C93E1
:102860008CE0481A8827580A2C96089581E00E9427
:10287000FF26A8EAB0E088278C9381E0A881B9817F
:102880008C93A881B9810C91083018F011F00C9448
:102890007014A881B981AD90BB24A4E8B0E0AA0D62
:1028A000BB1D0C91003211F40C946814A881B981FD
:1028B000AD90BB24A4E8B0E0AA0DBB1D8C91A8EAA2
:1028C000B0E08F930E9460268F918D9388278C9320
:1028D000A881B9818C918F5F8C9310F40C94411472
:1028E000A8EAB0E00E946026E0ECF0E50E94322702
:1028F00089E0A881B9818C93A881B9810C910B30B2
:1029000018F011F00C949E14A881B981AD90BB24ED
:10291000A4E8B0E0AA0DBB1D8C91A8EAB0E08F93AB
:102920000E9460268F918D9388278C93A881B9810E
:102930008C918F5F8C9310F40C947C1481E0481A76
:102940008827580A2296089581E00E94FF2681E098
:102950000E94FF2684E00E94FF268FEF0E94E3265C
:102960000E94E5260E94E426AC81BD818C938FEF06
:102970000E94E3260E94E5260E94E426AA81BB81EC
:102980008C93AA81BB810C9111272227332740E029
:1029900051E060E070E00E940F27A885B9850D9393
:1029A0001D932D933D93A885B9850D911D912D9172
:1029B0003C91AC81BD814C915527662777270E94B9
:1029C0008627A885B9850D931D932D933D93A885E2
:1029D000B9850D911D912D913C9140E050E061E051
:1029E00070E00E940F27A881B9810D931D932D934C
:1029F0003D938FEF0E94E3260E94E5260E94E42685
:102A0000AC81BD818C938FEF0E94E3260E94E52666
:102A10000E94E426AC81BD818C938FEF0E94E32657
:102A20000E94E5260E94E426AC81BD818C938FEF45
:102A30000E94E3260E94E5260E94E426AC81BD8127
:102A40008C938FEF0E94E3260E94E5260E94E426E5
:102A5000AC81BD818C938FEF0E94E3260E94E52616
:102A60000E94E426AA81BB818C93AA81BB810C9130
:102A700011272227332740E051E060E070E00E94F8
:102A80000F27A885B9850D931D932D933D93A88598
:102A9000B9850D911D912D913C91AC81BD814C91D9
:102AA0005527662777270E948627A885B9850D9325
:102AB0001D932D933D93A885B9850D911D912D9161
:102AC0003C91A881B9814D915D916D917C910E945D
:102AD0008627A885B9850D931D932D933D938FEF80
:102AE0000E94E3260E94E5260E94E426AC81BD8177
:102AF0008C938FEF0E94E3260E94E5260E94E42635
:102B0000AA81BB818C93AA81BB810C9111272227BA
:102B1000332740E051E060E070E00E940F27A88179
:102B2000B9810D931D932D933D93A881B9810D918A
:102B30001D912D913C91AC81BD814C91552766270B
:102B400077270E948627A881B9810D931D932D9325
:102B50003D938FEF0E94E3260E94E5260E94E42623
:102B6000AC81BD818C938FEF0E94E3260E94E52605
:102B70000E94E426AA81BB818C93AA81BB810C911F
:102B800011272227332740E051E060E070E00E94E7
:102B90000F27AE81BF810D931D932D933D93AE8181
:102BA000BF810D911D912D913C91AC81BD814C91C6
:102BB0005527662777270E948627AE81BF810D9310
:102BC0001D932D933D93AE81BF810D911D912D914C
:102BD0003C9140E050E061E070E00E940F27AE8140
:102BE000BF810D931D932D933D93AE81BF810D91B8
:102BF0001D912D913C91A881B9814D915D916D916F
:102C00007C910E948627AE81BF810D931D932D93E9
:102C10003D9386E0481A8827580A2696089584E04E
:102C20000E94FF2684E00E94FF26AC81BD810D91A9
:102C30001D912D913C9142E050E060E070E00E94D7
:102C40008B27A881B9810D931D932D933D93A3E705
:102C5000B0E00C91112722273327A881B9814D912B
:102C60005D916D917C910E940F27AA81BB810D938C
:102C70001D932D933D93AA81BB810D911D912D91A3
:102C80003C91AAE7B0E04D915D916D917C910E94DD
:102C90008627AA81BB810D931D932D933D930091AF
:102CA00082000B3011F40C946716AA81BB810D9140
:102CB0001D912D913C9140E250E060E070E00E9457
:102CC0008627AA81BB810D931D932D933D93AA81E5
:102CD000BB810D911D912D913C91AE81BF810D93D2
:102CE0001D932D933C9388E0481A8827580A249610
:102CF000089584E00E94FF2682E00E94FF26009152
:102D000082000B3011F00C94BD16AC81BD810D9189
:102D10001D912D913C9140E850E060E070E00E94F0
:102D20007026A5EDB0E04D935D936D937D93AC81DE
:102D3000BD810D911C9140E850E00E944626A8817B
:102D4000B9810D931C93A881B9810D911C9144E028
:102D500050E00E940527A881B9810D931C93A8819A
:102D6000B9810D911C9144E050E0040F151FA8811A
:102D7000B9810D931C930C94F316AC81BD810D9118
:102D80001D912D913C9140E051E060E070E00E9487
:102D90007026A5EDB0E04D935D936D937D93AC816E
:102DA000BD810D911C9140E051E00E944626A88112
:102DB000B9810D931C93A881B9810D911C9142E0BA
:102DC00050E00E940527A881B9810D931C93A8812A
:102DD000B9810D911C9142E050E0040F151FA881AC
:102DE000B9810D931C93A5EDB0E00D911D912D912E
:102DF0003C91AEE7B0E04D915D916D917C910E9468
:102E00008627A5EDB0E00D931D932D933D93A5ED81
:102E1000B0E00D911D912D913C91A1E7B0E04D9155
:102E20005C91662777270E948627A5EDB0E00D9379
:102E30001D932D933D930E94C91EA881B981AD9029
:102E4000BC90ADEDB0E0AA0DBB1D8C91AA81BB81F9
:102E50008D9388278D938D938C93A881B9810E943F
:102E6000F825AA81BB810D911D912D913C9140E0E7
:102E700051E060E070E00E940F27AA81BB810D93B2
:102E80001D932D933D93AA81BB810D911D912D9191
:102E90003C91A881B981AD90BC90ADEDB0E0AA0D98
:102EA000BB1D4C915527662777270E948627AA814C
:102EB000BB810D931D932D933D93009182000B30A8
:102EC00011F00C94C317A881B9810E94F825AA813A
:102ED000BB810D911D912D913C9140E051E060E04E
:102EE00070E00E940F27AA81BB810D931D932D9343
:102EF0003D93AA81BB810D911D912D913C91A8819B
:102F0000B981AD90BC90ADEDB0E0AA0DBB1D4C9168
:102F10005527662777270E948627AA81BB810D93B4
:102F20001D932D933D93A881B9810E94F825AA8114
:102F3000BB810D911D912D913C9140E051E060E0ED
:102F400070E00E940F27AA81BB810D931D932D93E2
:102F50003D93AA81BB810D911D912D913C91A8813A
:102F6000B981AD90BC90ADEDB0E0AA0DBB1D4C9108
:102F70005527662777270E948627AA81BB810D9354
:102F80001D932D933D93AA81BB810D911D912D9190
:102F90003C91AE81BF810D931D932D933C9386E0B0
:102FA000481A8827580A2496089580E0A881B98194
:102FB0008C930027BB27A0E38C9183FB0EF401E0E8
:102FC00040E0041711F00C94E91782E0A881B98160
:102FD0008C930027BB27A0E38C9184FB0EF401E0C7
:102FE00040E0041711F00C94F91781E0A881B98131
:102FF0008C930027BB27A3E38C9181FB0EF401E0A7
:1030000040E0041711F00C94091883E0A881B981FD
:103010008C930027BB27A3E38C9181FB0EF401E086
:1030200040E0041781E009F080E08F930027BB2780
:10303000A0E38C9183FB0EF401E040E0041781E0F3
:1030400009F080E09F918923882311F40C942C18B7
:1030500084E0A881B9818C93089581E00E94FF26C5
:1030600081E00E94FF2682E00E94FF265398549838
:1030700080E081BB909A919AEF93FF93E0EFF1E0AB
:103080000E94C426FF91EF9180E0AC81BD818C93BA
:103090000027BB27A0E38C9180FB0EF401E040E009
:1030A000041711F00C94581881E0AC81BD818C9309
:1030B0000027BB27A0E38C9181FB0EF401E040E0E8
:1030C000041711F00C946918AC81BD818C918E5F4E
:1030D0008C930027BB27A9E38C9185FB0EF401E0BC
:1030E00040E0041711F00C947A18AC81BD818C91EA
:1030F0008C5F8C930027BB27A9E38C9184FB0EF493
:1031000001E040E0041711F00C948B18AC81BD81F4
:103110008C91885F8C93AC81BD810C91003018F04C
:1031200011F00C9495180C94EE1885E090E00E9434
:10313000F02680E0AA81BB818C930027BB27A0E307
:103140008C9180FB0EF401E040E0041711F00C9428
:10315000AD1881E0AA81BB818C930027BB27A0E337
:103160008C9181FB0EF401E040E0041711F00C9407
:10317000BE18AA81BB818C918E5F8C930027BB27E0
:10318000A9E38C9185FB0EF401E040E0041711F0F7
:103190000C94CF18AA81BB818C918C5F8C930027F3
:1031A000BB27A9E38C9184FB0EF401E040E00417F7
:1031B00011F00C94E018AA81BB818C91885F8C93EC
:1031C000AA81BB814C91AC81BD810C91041711F493
:1031D0000C94EE1880E0AC81BD818C93AC81BD81F4
:1031E0000C91033011F00C94FB1882E0AC81BD818E
:1031F0008C930C943119AC81BD810C91043081E029
:1032000008F480E08F93AC81BD810C91073081E0A0
:1032100010F009F080E09F918923882311F40C9429
:10322000171983E0AC81BD818C930C943119AC816A
:10323000BD810C91083081E008F480E08F93AC816F
:10324000BD810C910F3081E010F009F080E09F917A
:103250008923882311F40C94311984E0AC81BD8159
:103260008C9381E081BB9198539A549AAC81BD8133
:103270008C91AE81BF818C9384E0481A8827580ACC
:103280002696089581E00E94FF2681E00E94FF2695
:10329000AC81BD818C91A881B9818C930E94EF088B
:1032A00088EC90E00E94F0265A924A9281E0A42D88
:1032B000B52D8C9381E00E94DE250E943F2322964B
:1032C00081E00E94DA25A895EBE6F0E0FA93EA9314
:1032D0000E94D51722968AE090E00E94F026009185
:1032E0006B00003011F00C94631986E990E00E94A5
:1032F000F0265A924A9280E0A42DB52D8C9381E05D
:103300000E94DE250E943F23229681E00E94DA255A
:1033100084E690E00E94F0265A924A9280E0A42D22
:10332000B52D8C9381E00E94DE250E943F232296DA
:1033300081E00E94DA25A895EBE6F0E0FA93EA93A3
:103340000E94D51722960E94F1085A924A9281E073
:10335000A42DB52D8C9381E00E94DE250E943F2391
:10336000229681E00E94DA2584E690E00E94F02611
:103370005A924A9280E0A42DB52D8C9381E00E9450
:10338000DE250E943F23229681E00E94DA258AE012
:1033900090E00E94F0265A924A9280E0A42DB52D2A
:1033A0008C9381E00E94DE250E943F23229681E0DB
:1033B0000E94DA250E94EF0886E990E00E94F0263C
:1033C00000916B00003018F011F00C94E9190C9486
:1033D0009B1988E790E00E94F0265A924A9281E079
:1033E000A42DB52D8C9381E00E94DE250E94001B48
:1033F000229681E00E94DA25A881B9810C910230E1
:1034000011F00C94431A00916B00013011F00C94F0
:103410000E1A81E08093C5000C943C1A023011F022
:103420000C94261A80E08093C5005A924A9281E05B
:10343000A42DB52D8C9381E00E94DE250E94001BF7
:10344000229681E00E94DA250C943C1A033011F098
:103450000C943C1A83E08093C5005A924A9282E011
:10346000A42DB52D8C9381E00E94DE250E94001BC7
:10347000229681E00E94DA25EEE0F0E0A5ECB0E0D3
:103480007BE70E941928A881B9810C91033011F0C3
:103490000C946C1A00916B00013011F00C94551AC9
:1034A00081E0809370000C94651A023011F00C9446
:1034B0005E1A80E0809370000C94651A033011F05E
:1034C0000C94651A82E080937000E1E1F0E0A0E7DF
:1034D000B0E07BE70E941928A881B9810C910130E6
:1034E00011F00C94BE1A00916B00013011F00C9495
:1034F000851AA6ECB0E08C91897F8C93A6ECB0E0A5
:103500008C9182608C930C94B71A023011F00C9459
:103510009F1AA6ECB0E08C91897F8C935A924A92C4
:1035200081E0A42DB52D8C9381E00E94DE250E94C0
:10353000001B229681E00E94DA250C94B71A033012
:1035400011F00C94B71AA6ECB0E08C9186608C93C5
:103550005A924A9284E0A42DB52D8C9381E00E946A
:10356000DE250E94001B229681E00E94DA25EFE012
:10357000F0E0A6ECB0E07BE70E9419280E94F30877
:10358000A895EBE6F0E0FA93EA930E94D51722960D
:1035900085E090E00E94F02600916B00003011F071
:1035A0000C94C01A86E990E00E94F0265A924A9242
:1035B00080E0A42DB52D8C9381E00E94DE250E9431
:1035C0003F23229681E00E94DA2586E990E00E945E
:1035D000F0265A924A9280E0A42DB52D8C9381E07A
:1035E0000E94DE250E943F23229681E00E94DA2578
:1035F0000E94F10882E0481A8827580A2496089504
:1036000081E00E94FF2681E0A881B9818C93AA8184
:10361000BB814C91A881B9810C91041718F011F06D
:103620000C942D1B5A924A9282E0A42DB52D8C93B6
:1036300081E00E94DE250E943F23229681E00E94C5
:10364000DA258DE790E00E94F026A881B9818C915F
:103650008F5F8C9310F40C94071B81E0481A882725
:10366000580A2296089581E00E94FF2681E0A881F1
:10367000B9818C93A881B9810C91063018F011F0B2
:103680000C94561B0E94EF088FE090E00E94F026F9
:103690000E94F10884E690E00E94F026A881B9819A
:1036A0008C918F5F8C9310F40C943A1B81E0481A34
:1036B0008827580A229608950E94DC26C39A88EC2F
:1036C00090E00E94F02681B5886081BD0E940122B1
:1036D0005A924A9281E0A42DB52D8C9381E00E94EC
:1036E000DE250E944D22229681E00E94DA2581B5D6
:1036F000886181BD877F81BD84E690E00E94F026CD
:10370000FF27E0E1FA93EA935A924A928BE0A42DC4
:10371000B52D8C9381E00E94DE250E94E42424963E
:1037200081E00E94DA25013051E0150711F00C9478
:10373000AC1B5A924A92A0ECB0E08D919C91A42DC2
:10374000B52D8D939C9382E00E94DE250E94E52298
:10375000229682E00E94DA255A924A9282E3A42DB0
:10376000B52D8C9381E00E94DE250E944D22229689
:1037700081E00E94DA25C29AD89A82E390E00E9402
:10378000F026089581E00E94FF2681E00E94FF2636
:103790008FEFAA81BB818C9380E0A881B9818C9343
:1037A000A881B9810C910F3018F011F00C94E51B31
:1037B00091E0AA81BB810E94D226A881B9818C9117
:1037C0008F5F8C9310F40C94D01B82E0481A8827EA
:1037D000580A2496089581E00E94FF2681E00E9405
:1037E000FF2681E00E94FF2682E00E94FF2682E001
:1037F0000E94FF268FEFAA85BB858C93C49A0E94F6
:10380000C21BC498EE81FF81FA93EA935A924A92BE
:1038100080E4A42DB52D8C9381E00E94DE255A9280
:103820004A9200E010E020E030E0A42DB52D0D9389
:103830001D932D933C9384E00E94DE250E94752108
:10384000269685E00E94DA25AE81BF810C91013079
:1038500011F40C942E1CC49A0C94C31E81E0AA850A
:10386000BB858C9380E293E0A881B9818D939C9372
:10387000EE81FF81FA93EA935A924A9287E7A42D48
:10388000B52D8C9381E00E94DE255A924A9200E089
:1038900010E020E030E0A42DB52D0D931D932D9365
:1038A0003C9384E00E94DE250E947521269685E0E7
:1038B0000E94DA2581E090E00E94F026EE81FF81EF
:1038C000FA93EA935A924A9289E6A42DB52D8C93E5
:1038D00081E00E94DE255A924A9200E010E020E04A
:1038E00030E0A42DB52D0D931D932D933C9384E0D2
:1038F0000E94DE250E947521269685E00E94DA2529
:1039000081E090E00E94F026AE81BF810C910030F2
:1039100081E009F080E08F93AE81BF810C9105308A
:1039200081E009F080E09F91892B8F93A881B98174
:103930000D911C91003050E0150781E009F080E006
:103940009F91892B882311F40C94381CAE81BF8180
:103950000C91003011F00C94B01CC49A0C940D1D05
:1039600080E293E0A881B9818D939C93EE81FF81E1
:10397000FA93EA935A924A9281E4A42DB52D8C933E
:1039800081E00E94DE255A924A9200E010E020E099
:1039900030E0A42DB52D0D931D932D933C9384E021
:1039A0000E94DE250E947521269685E00E94DA2578
:1039B000A881B9810D911C9141E050E0041B150BC9
:1039C000A881B9810D931C9381E090E00E94F026BC
:1039D000AE81BF810C91003081E009F080E08F93CF
:1039E000A881B9810D911C91003050E0150781E04C
:1039F00009F080E09F91892B882311F40C94B61C68
:103A0000C49AA881B9810D911C91003050E015072E
:103A100011F00C940D1D0C94C31E8AE090E00E94DE
:103A2000F026C498EE81FF81FA93EA935A924A9263
:103A300080E5A42DB52D8C9381E00E94DE255A925D
:103A40004A9201E010E020E030E0A42DB52D0D9366
:103A50001D932D933C9384E00E94DE250E947521E6
:103A6000269685E00E94DA25C49A82E390E00E94BF
:103A7000F02600E010E020E030E0AEE7B0E00D938B
:103A80001D932D933C9300E010E020E030E0A5ED85
:103A9000B0E00D931D932D933C930E94C91E00E04E
:103AA00010E020E030E0A5EDB0E00D931D932D93E4
:103AB0003C930027A3EDB0E08C9186FB0EF401E06F
:103AC00041E0041711F00C94671D0C94C31E009183
:103AD000EA00023011F40C94FA1D8091A002809348
:103AE0008200A7EAB2E00D91112740E051E00E9468
:103AF0000527AA81BB810D931C93AA81BB810D91DF
:103B00001C91A6EAB2E04D915527040F151FAA811A
:103B1000BB810D931C93AA81BB810D911C9122271F
:103B2000332740E050E061E070E00E940F27AEE7ED
:103B3000B0E00D931D932D933D93A5EAB2E00D9156
:103B4000112740E051E00E940527AA81BB810D9317
:103B50001C93AA81BB810D911C91A4EAB2E04D9106
:103B60005527040F151FAA81BB810D931C93AEE747
:103B7000B0E00D911D912D913C91AA81BB814D9199
:103B80005C91662777270E948627AEE7B0E00D9309
:103B90001D932D933D93009182000C3011F00C94F5
:103BA000D41D8BE080938200009182000E3011F0D2
:103BB0000C94DD1D8BE080938200009182000F3019
:103BC00011F00C94E61D8BE080938200AEE7B0E02C
:103BD0000D911D912D913C91A5EDB0E00D931D939C
:103BE0002D933C930E94C91EA5EDB0E00E94FF25D5
:103BF0000C940C1E00911401063411F00C94031E59
:103C000084E08093820000913001063411F00C941E
:103C10000C1E8BE080938200A8958091EB0080932E
:103C2000730000917300003011F00C94191E0C9475
:103C3000C31E00917300003418F011F00C94221E82
:103C40000C94241E0C94C31E8091EC00AE81BF81A5
:103C50008C938091ED00AC81BD818C93AC81BD8152
:103C60009C91AE81BF818C91A1E7B0E08D939C9334
:103C70008091F400AE81BF818C938091F500AC817E
:103C8000BD818C93AC81BD819C91AE81BF818C91B3
:103C9000A4E7B0E08D939C93A4E7B0E00D911C9154
:103CA000003050E0150711F00C946C1E8091020159
:103CB000AE81BF818C9380910301AC81BD818C93D7
:103CC000AC81BD819C91AE81BF818C91A4E7B0E0B5
:103CD0008D939C930C946C1EA895A4E7B0E00D9175
:103CE0001C91003050E0150711F00C94791E0C94D3
:103CF000C31E02E010E020E030E0A4E7B0E04D9108
:103D00005C91662777270E940F27A6E7B0E00D9306
:103D10001D932D933D93A6E7B0E00D911D912D913C
:103D20003C91A1E7B0E04D915C91662777270E9416
:103D30008627A6E7B0E00D931D932D933D93A6E74C
:103D4000B0E00D911D912D913C91A5EDB0E04D910C
:103D50005D916D917C910E948627A6E7B0E00D935E
:103D60001D932D933D93A6E7B0E00D911D912D91EC
:103D70003C91A5EDB0E00D931D932D933C9380E015
:103D8000AA85BB858C9387E0481A8827580A2A960B
:103D9000089581E00E94FF2681E00E94FF2682E0D4
:103DA0000E94FF2682E00E94FF268FEFAE81BF8136
:103DB0008C9391E0AE81BF810E94D22691E0AE81CA
:103DC000BF810E94D22691E0AE81BF810E94D2269F
:103DD00091E0AE81BF810E94D22691E0AE81BF8189
:103DE0000E94D22691E0AE81BF810E94D22691E04E
:103DF000AE81BF810E94D22691E0AE81BF810E9438
:103E0000D22691E0AE81BF810E94D22691E0AE81A0
:103E1000BF810E94D22691E0AE81BF810E94D2264E
:103E200091E0AE81BF810E94D22691E0AE81BF8138
:103E30000E94D22691E0AE81BF810E94D22691E0FD
:103E4000AE81BF810E94D22691E0AE81BF810E94E7
:103E5000D226C49880E090E0A881B9818D939C938C
:103E60008FEF0E94E3260E94E5260E94E426AE81A1
:103E7000BF818C93A881B9810E94F125AE81BF8159
:103E80000C91003081E009F480E08F93A881B98122
:103E90000D911C91003050E0150781E009F080E0A1
:103EA0009F91892B882311F40C94301FA881B9812C
:103EB0000D911C91003050E0150711F00C94671F14
:103EC0008091D30080648093D3000C948C20EE8189
:103ED000FF81FA93EA935A924A9281E5A42DB52D77
:103EE0008C9381E00E94DE255A924A92A5EDB0E0C3
:103EF0000D911D912D913C91A42DB52D0D931D93E8
:103F00002D933C9384E00E94DE250E947521269625
:103F100085E00E94DA250027A3EDB0E08C9186FBB6
:103F20000EF401E041E0041711F00C94991F0C9479
:103F30008C20A895AE81BF810C91003011F00C94BB
:103F4000DE1F80E090E0A881B9818D939C938FEF74
:103F50000E94E3260E94E5260E94E426AE81BF81EE
:103F60008C93A881B9810E94F125AE81BF810C910B
:103F7000003081E009F480E08F93A881B9810D9130
:103F80001C91003050E0150781E009F080E09F911E
:103F9000892B882311F40C94A71FA881B9810D9156
:103FA0001C91003050E0150711F00C94DE1F809139
:103FB000D30080648093D3000C948C20AE81BF81A9
:103FC0000C910F3F11F00C94222080E090E0A8812A
:103FD000B9818D939C938FEF0E94E3260E94E52682
:103FE0000E94E426AE81BF818C93A881B9810E9492
:103FF000F125AE81BF810C910F3F81E009F480E093
:104000008F93A881B9810D911C91003050E0150764
:1040100081E009F080E09F91892B882311F40C94B2
:10402000EB1FA881B9810D911C91003050E015075C
:1040300011F00C9422208091D30080648093D300EF
:104040000C948C20AE81BF810C910E3F11F40C9426
:104050003120C49A8091D30080648093D3000C9463
:104060008C2080E090E0AA81BB818D939C9380E0BE
:10407000AE81BF818C93AE81BF810C910F3F18F050
:1040800011F00C947320AA81BB810E94F1258FEF5F
:104090000E94E3260E94E5260E94E426AA81BB81B5
:1040A000AD90BC90ADEDB0E0AA0DBB1D8C93AA8184
:1040B000BB810E94F1258FEF0E94E3260E94E52636
:1040C0000E94E426AA81BB81AD90BC90ADEDB0E02A
:1040D000AA0DBB1D8C93AE81BF818C918F5F8C9399
:1040E00010F40C943B208FEF0E94E3260E94E526FB
:1040F0000E94E426AE81BF818C938FEF0E94E3265D
:104100000E94E5260E94E426AE81BF818C93C49A6A
:10411000A5EDB0E00E94E22586E0481A8827580AFB
:104120002896089582E00E94FF2681E00E94FF26E3
:1041300080E0AE81BF818C930E94C21BC49880E056
:1041400090E0AA81BB818D939C938FEF0E94E32620
:104150000E94E5260E94E426A881B9818C93AA8159
:10416000BB810E94F125A895A881B9810C910030EE
:1041700081E009F480E08F93AA81BB810D911C91AD
:10418000003050E0150781E009F080E09F91892B15
:10419000882311F40C94A520AA81BB810D911C9158
:1041A000003050E0150711F00C94DD208091D30011
:1041B00080648093D3000C946F21E881F981FA9395
:1041C000EA935A924A9281E5A42DB52D8C9381E011
:1041D0000E94DE255A924A92AA85BB850D911D91B7
:1041E0002D913C91A42DB52D0D931D932D933C93B2
:1041F00084E00E94DE250E947521269685E00E94BB
:10420000DA25A881B9810C91003011F00C94352188
:1042100080E090E0AA81BB818D939C938FEF0E94F8
:10422000E3260E94E5260E94E426A881B9818C93AA
:10423000AA81BB810E94F125A895A881B9810C9122
:10424000003081E009F480E08F93AA81BB810D9159
:104250001C91003050E0150781E009F080E09F914B
:10426000892B882311F40C940E21A881B9810C911B
:104270000F3F11F00C94692180E090E0AA81BB818E
:104280008D939C938FEF0E94E3260E94E5260E9467
:10429000E426A881B9818C93AA81BB810E94F12573
:1042A000A895A881B9810C910F3F81E009F480E0C5
:1042B0008F93AA81BB810D911C91003050E01507AE
:1042C00081E009F080E09F91892B882311F40C9400
:1042D0004221A881B9818C91AE81BF818C9383E00A
:1042E000481A8827580A2496089584E00E94FF26D9
:1042F00081E00E94FF2682E00E94FF268FEFAA81C4
:10430000BB818C9391E0AA81BB810E94D22691E06F
:10431000A885B9850E94D226AE81BF810D911D91DD
:104320002D913C9140E052E060E070E00E940F2748
:10433000AC81BD810D931D932D933D93AC81BD81C7
:104340008F9314968E910E94F6218E910E94F621F1
:104350008E910E94F6218E910E94F62185E90E949D
:10436000F6218F9180E090E0A881B9818D939C9394
:104370008FEF0E94E3260E94E5260E94E426AA8190
:10438000BB818C93A881B9810E94F125A895AA814F
:10439000BB810C910F3F81E009F480E08F93A881ED
:1043A000B9810D911C91003050E0150781E009F0B2
:1043B00080E09F91892B882311F40C94B821A88167
:1043C000B9810D911C91003050E0150711F00C944B
:1043D000EE218091D30080648093D300AA81BB81B9
:1043E0008C91AA85BB858C930C94FB218FB9779B0C
:1043F000FECF8FB1089587E0481A8827580A26967D
:1044000008955A924A9284E298E0A42DB52D8D9396
:104410009C9382E00E94DE255A924A9280E0A42D6D
:10442000B52D8C9381E00E94DE250E94892424967C
:1044300083E00E94DA25EF93FF93ECE8F1E00E941D
:10444000C426FF91EF91BB27A0E38C9182FBDEF79E
:1044500082E090E00E94F0265A924A9280E298E030
:10446000A42DB52D8D939C9382E00E94DE255A9257
:104470004A9280E0A42DB52D8C9381E00E94DE2528
:104480000E948924249683E00E94DA2582E090E04D
:104490000E94F0260E940223089582E00E94FF26D7
:1044A00000E011E0AA81BB814D9155270E940527AC
:1044B000A881B9810D931C93A881B9810D911C919C
:1044C000AA81BB814D915527040F151FA881B98181
:1044D0000D931C935A924A92AA81BB818D919C9113
:1044E000A42DB52D8D939C9382E00E94DE255A92D7
:1044F0004A928BE0A42DB52D8C9381E00E94DE259D
:104500000E948924249683E00E94DA255A924A92D6
:1045100080E298E0A42DB52D8D939C9382E00E94BB
:10452000DE255A924A9280E0A42DB52D8C9381E02D
:104530000E94DE250E948924249683E00E94DA25C9
:1045400082E0481A8827580A2296089582E00E943D
:10455000FF2600E110E0AC81BD814D9155270E94FE
:104560000527A881B9810D931C93A881B9810D916C
:104570001C91AA81BB814D915527040F151FA8815D
:10458000B9810D931C935A924A92AA81BB818D9155
:104590009C91A42DB52D8D939C9382E00E94DE25E5
:1045A0005A924A9282E0A42DB52D8C9381E00E940C
:1045B000DE250E948924249683E00E94DA2582E089
:1045C000481A8827580A229608955A924A92AA8130
:1045D000BB818D919C91A42DB52D8D939C9382E0F0
:1045E0000E94DE255A924A9283E0A42DB52D8C9329
:1045F00081E00E94DE250E948924249683E00E94A7
:10460000DA25089581E00E94FF2681E00E94FF26BE
:10461000C49AD898C29880E0A881B9818C9380E030
:10462000AA81BB818C93AA81BB810C910F3118F0B8
:1046300011F00C94372391E0A881B9810E94D22611
:1046400091E0A881B9810E94D22691E0A881B98128
:104650000E94D22691E0A881B9810E94D226AA8127
:10466000BB818C918F5F8C9310F40C941323C29AAE
:10467000D89A82E0481A8827580A2496089581E03B
:104680000E94FF265A924A9280E298E0A42DB52D0E
:104690008D939C9382E00E94DE255A924A9280E09C
:1046A000A42DB52D8C9381E00E94DE250E948924E3
:1046B000249683E00E94DA25AA81BB810C91003008
:1046C00011F00C9472235A924A9280E0A42DB52DD9
:1046D0008C9381E00E94DE250E94EC23229681E0EB
:1046E0000E94DA25AA81BB810C91013011F00C9453
:1046F00088235A924A9285E6A42DB52D8C9381E0A9
:104700000E94DE250E94EC23229681E00E94DA2599
:10471000AA81BB810C91023011F00C94B5235A92FE
:104720004A9283E6A42DB52D8C9381E00E94DE256C
:104730000E94EC23229681E00E94DA2588EC90E02A
:104740000E94F0265A924A9280E0A42DB52D8C93B7
:1047500081E00E94DE250E94EC23229681E00E94E7
:10476000DA2582E390E00E94F026AA81BB810C91B9
:10477000033011F00C94DE235A924A9282E6A42D63
:10478000B52D8C9381E00E94DE250E94EC232296B9
:1047900081E00E94DA2580E991E00E94F0265A9299
:1047A0004A9280E0A42DB52D8C9381E00E94DE25F5
:1047B0000E94EC23229681E00E94DA258AE090E0B4
:1047C0000E94F0268AE090E00E94F02681E0481ADC
:1047D0008827580A2296089581E00E94FF26C49AED
:1047E0005A924A928CE3A42DB52D8C9381E00E94BD
:1047F000DE250E944D22229681E00E94DA25D8987B
:10480000C298AA81BB810C91003018F011F00C9471
:104810000B240C94452483E5A881B9818C9391E005
:10482000A881B9810E94D2268FEEA881B9818C938C
:1048300091E0A881B9810E94D2268EE6A881B98133
:104840008C9391E0A881B9810E94D22691E0AA813F
:10485000BB810E94D22680E0A881B9818C9391E02F
:10486000A881B9810E94D22691E0A881B9810E94D5
:10487000D22691E0A881B9810E94D22691E0A88138
:10488000B9810E94D2260C94812485E4A881B98143
:104890008C9391E0A881B9810E94D22688E7A881F3
:1048A000B9818C9391E0A881B9810E94D22689E6D2
:1048B000A881B9818C9391E0A881B9810E94D22608
:1048C00084E7A881B9818C9391E0A881B9810E9485
:1048D000D22680E0A881B9818C9391E0A881B9812A
:1048E0000E94D22691E0A881B9810E94D22691E04F
:1048F000A881B9810E94D22691E0A881B9810E9445
:10490000D226C29AD89A81E0481A8827580A229655
:10491000089581E00E94FF26C29AD8985A924A923E
:1049200082E0A42DB52D8C9381E00E94DE250E94AB
:104930003E25229681E00E94DA255A924A92AC8165
:10494000BD818C91A42DB52D8C9381E00E94DE2534
:104950000E943E25229681E00E94DA25AC81BD812D
:1049600011968C91A881B9818C935A924A92AA810E
:10497000BB818C91A42DB52D8C9381E00E94DE2506
:104980000E943E25229681E00E94DA25AC81BD81FD
:104990008C91A881B9818C935A924A92AA81BB8149
:1049A0008C91A42DB52D8C9381E00E94DE250E9470
:1049B0003E25229681E00E94DA25D89A81E0481AA5
:1049C0008827580A2296089581E00E94FF2681E0F8
:1049D0000E94FF2682E00E94FF26C29AD8985A922F
:1049E0004A9283E0A42DB52D8C9381E00E94DE25B0
:1049F0000E943E25229681E00E94DA255A924A9230
:104A0000A885B9858C91A42DB52D8C9381E00E9449
:104A1000DE250E943E25229681E00E94DA25EC8167
:104A2000FD81FA93EA930E9444252296EA81FB8154
:104A3000FA93EA930E9444252296D89AAC81BD81CC
:104A40000D91112740E051E00E940527A881B9810E
:104A50000D931C93A881B9810D911C91AA81BB81F2
:104A60004D915527040F151FA885B9850D931C93EB
:104A700084E0481A8827580A2696089591E0A8816C
:104A8000B9810E94D226089581E00E94FF2691E01C
:104A9000A881B9810E94C726A881B9818C91AA8179
:104AA000BB818C9381E0481A8827580A2296089582
:104AB00082E00E94FF2681E00E94FF26C49ABB2765
:104AC000A0E38C9182FBDEF7C298AC81BD810D9191
:104AD0001C91003052E0150711F00C94A72581E0DD
:104AE00090E0AA81BB818D939C9380E0A881B981DD
:104AF0008C93A881B9810C910F3018F011F00C94AF
:104B0000A525BB27A0E38C9182FBDEF790E2AA816A
:104B1000BB81AD90BC90ADEDB0E0AA0DBB1D0E9475
:104B2000D226AA81BB810D911C9140E250E0040F76
:104B3000151FAA81BB810D931C93A881B9818C910B
:104B40008F5F8C9310F40C9479250C94D32581E01D
:104B500090E0AA81BB818D939C93AC81BD814D91E6
:104B60005C91AA81BB810D911C910417150718F067
:104B700011F00C94D325BB27A0E38C9182FBDEF7C8
:104B8000C29A91E0AA81BB81AD90BC90ADEDB0E03E
:104B9000AA0DBB1D0E94D226AA81BB810E94F125CD
:104BA00010F40C94AD25C29A83E0481A8827580A5D
:104BB00024960895481A8827580A0895480E882789
:104BC000581E08950D911D912D913C9181E0080F83
:104BD0008827181F281F381F3C932E931E930E936F
:104BE0000895ED91FC91EF5FFF4FFC93EE930895D4
:104BF000ED91FC91E150F040FC93EE9308950D91FE
:104C00001D912D913C9101501040204030403C932B
:104C10002E931E930E9308954091DF025091E0026F
:104C20000DE815E30E94202649E156E3040F151F05
:104C30000093DF021093E002498158810C944626CC
:104C400009D00E94052700FC10D0089503D01ED083
:104C500001F8F9CF0024E89457FF02C009D0689406
:104C600000F80BD010F80124089502D009D008955F
:104C7000509540954F5F5F4F0895E89417FF089552
:104C8000009510950F5F1F4F68940895352F242FBE
:104C9000E894452B11F468940895512F402F002774
:104CA000112780E1440F551F001F111F021B130B1A
:104CB000416018F4020F131F4E7F8A9599F70895EB
:104CC0008F938D918823E9F711978F91089588EE3E
:104CD00093E086D03197D9F7089500FC05D0089568
:104CE00030D005D001F8F9CF37D03FD00895842FC8
:104CF000952FA62FB72FE894452B462B472B11F461
:104D000068940895402F512F622F732F0027112789
:104D100022273327F0E2440F551F661F771F001F1D
:104D2000111F221F331F081B190B2A0B3B0B41605D
:104D300028F4080F191F2A1F3B1F4E7FFA9559F7B9
:104D400008950024E89477FF02C006D0689400F824
:104D500009D010F80124089512D04F5F5F4F6F4FB4
:104D60007F4F0895E89437FF08950095109520959A
:104D700030950F5F1F4F2F4F3F4F68940895409518
:104D800050956095709508953197F1F708950E94B8
:104D9000E3268C910E94E5268D939A95D1F70E9487
:104DA000E42608950E94E3268D910E94E5269A95B7
:104DB000D9F70E94E4260895BF9ABE98C69ABD9A74
:104DC00080E58DB90895089508958FB9779BFECF3A
:104DD0008FB10895689462F80895E89462F8089590
:104DE000EF93FF93EE27E82BE92B31F0E0EDF7E0AE
:104DF0003197F1F70197D1F7FF91EF9108955A920A
:104E00004A92480E8827581E08950F92B801469F6F
:104E10008001479F100D569F100D0F9008950F921F
:104E20001F922F92C801D901489F80014A9F90018B
:104E30004B9F202C499F100D211D321D5A9F202C65
:104E4000589F100D211D321D599F200D311D689F47
:104E5000200D311D699F300D789F300D2F901F90D0
:104E60000F9008950E9438270D920020D9F70895D9
:104E7000C895319600200895819104D08D938823A0
:104E8000D9F70895813618F08B3708F48F7D08958F
:104E90002E2E3F2E992781918D3209F093958823EC
:104EA000D1F79A95E22DF32D112361F0091718F02F
:104EB00011F0101B01C0191B28F021F080E28D9326
:104EC0001A95E9F780818D3219F48D93319604C0DB
:104ED000222311F08BE28D93091738F031F0091B72
:104EE00021F080E38D930A95E9F781918D938823D2
:104EF000E1F7332351F0EA2FFB2F319633958E9152
:104F000082933A95E1F78EE28C930895040F151F72
:104F1000261F371F0895041B150B260B370B08950A
:104F200004171507260737070895000F111F221FC2
:104F3000331F089500951095209530950F5F1F4FF2
:104F40002F4F3F4F0895019110810EC00191119193
:104F5000219130810BC00191108117FF05C03FEFF7
:104F60002FEF04C0008111272227332737FF03C00A
:104F7000E1DF8DE28D93CF93DF93CF92DF92EF92BB
:104F8000AA24BB24CC24DD24EE2440E2CAE0DD27A1
:104F900055E093E38881890F87FD9F7083FD907FA3
:104FA000891B89935A95A9F7C0DFAA1CBB1CCC1C8E
:104FB000DD1CEE1C4A9551F7E894EFE0FF27829143
:104FC0000ED0EB30E0F71EF068948A2D0CD08827C5
:104FD0008D93EF90DF90CF90DF91CF910895982F30
:104FE000829501D0892F8F70805D26F0803309F47F
:104FF000089568948D93089588278D9308958191DD
:105000008D938823E1F7089509919191992351F0A7
:105010008A95D9F7319781918D930A9519F0882354
:10502000D1F70895E9CFE199FECFEEBBFFBB3196F2
:10503000089591E001C092E07B3751F47FB7F89476
:10504000F2DF8D918DBBE29AE19A9A95C9F77FBF05
:105050007727089591E001C092E0E5DFE09A8DB3F3
:105060008D939A95D1F70895FF93881BF9E0001F5F
:10507000FA9511F4FF910895881F841B18F4840F8A
:105080008894F5CF0894F3CF689401C0E894AF9367
:10509000BF938D9116F0919103C00E943827902DF7
:1050A000891718F011F48823A1F7BF91AF910895E3
:1050B0004F005A0059004200434F4E4649470000F6
:0250C0002E00C0
:00000001FF
